:1018000022C040C059C03EC03DC03CC03BC03AC0F1
:1018100039C038C037C036C035C034C033C0090203
:1018200012000101008032090400000000000000E5
:1018300012011001FF000008D01653070601000036
:1018400000010403090411241FBECFE5D2E0DEBF6E
:10185000CDBF00EB0F9307E00F9310E0A0E6B0E0E0
:10186000E2ECFFE102C005900D92A636B107D9F770
:1018700020E0A6E6B0E001C01D92AB39B207E1F767
:10188000F0D19DC3BDCFA82FB92F80E090E041E0FB
:1018900050EA609530E009C02D9182279795879591
:1018A00010F084279527305EC8F36F5FA8F3089582
:1018B000EADF8D939D930895CF93CFB7CF93C091D7
:1018C0005F02C03B21F4C0915E02C73021F0CF918E
:1018D000CFBFCF9194CFCC27C395B39BE9F7B39BF0
:1018E0000BC0B39B09C0B39B07C0B39B05C0B39BA0
:1018F00003C0B39B01C0D3C00F92DF93C0917E00A1
:10190000DD27CB57DF4F012EB39B03C0DF910F9034
:10191000E6CF2F930F931F934F932FEF4F6F06B385
:1019200003FB20F95F933F9350E03BE065C016B3A3
:101930000126502953FDC89556B3012703FB25F90D
:101940002F7306B3B1F05027102713FB26F906B208
:101950002230F0F000C016B3012703FB27F901265F
:10196000502906B22430E8F54F77206816B30000FE
:10197000F6CF50274F7D206206B2102F000000C026
:1019800006B300265029102713FB26F906B2E2CF32
:101990004F7B06B3206400C0DACF012650291871AE
:1019A00006B269F14E7F2160012F16B328C00026D0
:1019B00050294D7F06B22260102F29C001265029E0
:1019C0004B7F06B22460012F2DC016B3012650298B
:1019D000477F2860000006B22EC04F7E06B320610C
:1019E00030C0422706B3499300265029102706B27B
:1019F0004FEF13FB20F9297F16B379F2187159F1D3
:101A00000126502906B2012703FB21F9237F06B3E3
:101A100071F2002650293150D0F006B2102713FB86
:101A200022F9277E16B351F201265029012703FB24
:101A300006B223F92F7C49F2000006B3102713FBEE
:101A400024F90026502906B22F7939F270CF10E21E
:101A50001ABF002717C03B503195C31BD04010E27E
:101A60001ABF0881033CF9F00B34E9F020917C00A7
:101A70001981110F1213EDCF093651F10D3211F00A
:101A8000013E39F7009383003F915F914F911F9181
:101A90000F912F91DF910F90CAB7C5FD1DCFCF9148
:101AA000CFBFCF91189520918300222369F3109125
:101AB0008100112321F5343022F1309381002093ED
:101AC0007D0010917E003BE0311B30937E0019C0F9
:101AD0000091810001309CF40AE53091600034FDF2
:101AE00011C000936000C1E7D0E010C0052710E0EE
:101AF00000C021C0052710E0C89508BB14C03AE516
:101B000001C032ED032EC0E0D0E032E017B318611F
:101B1000C39A08B317BB58E120E84FEF20FF052711
:101B200008BB279517951C3F28F700004552B0F7D2
:101B300020FF0527279508BB17951C3FB8F629916C
:101B40003A9561F7077E10918200110F08BBC250D1
:101B5000D04011F010937C0010E21ABF086017B358
:101B6000177E402F477E54E05A95F1F708BB17BB0C
:101B700048BB8ACFF8942FEFB0E8A0E44AE0B1BFA9
:101B8000000081EE9CE0B399FECFB39BFECF01979E
:101B9000B399FDCF97FF03C0BA1B819501C0BA0F5F
:101BA000A69529F4281710F031B7282FA1E041504D
:101BB00031F731BF0000789408958FB7F894E09121
:101BC0006900F0916A00329795E090935700E8958C
:101BD0008FBF08952091690030916A002115310569
:101BE00089F12430310591F12C3F47E1340739F474
:101BF00080916B0090916C008E5F9B4F10C02E3FC8
:101C000047E1340739F480916D0090916E008D5F4B
:101C10009B4F05C02A3F374111F481B790E02FB7A1
:101C2000F894E0916900F0916A0031E00C01309382
:101C30005700E89511242FBF3296F0936A00E09385
:101C40006900089581E180935700E8958FEF9BEC40
:101C5000E6CF8FEF9FEFBEDF809169008F73C9F7EA
:101C6000ACCF88E10FB6F89481BD11BC0FBEE1E0A6
:101C7000F0E0E491EF3F09F4ECDF10926A0010927B
:101C8000690086ED80936700C198AC9A8BB780623B
:101C90008BBFBB9A88EB9BE0ECE9F1E03197F1F761
:101CA0000197D1F7BB98789400918100035007FD0C
:101CB000CFC080917E00CCE0D0E0C81BD109CB57CB
:101CC000DF4F80917D008D3209F090C0083009F01F
:101CD000BDC083EC809371008AE580936000109210
:101CE0006F002881922F90768981992329F1109293
:101CF000670010926600811108C082E690E0909320
:101D0000800080937F0014E067C0813051F48C81A3
:101D10009D8190936A008093690027FD58C01FEF52
:101D200057C090916800823011F4916001C09460B6
:101D30009093680010E050C09A8110927A0081114F
:101D400006C010927B008AE790E012E03BC085302D
:101D500019F4909382002CC0863009F58B81813074
:101D600019F480E398E104C0823041F48EE198E1F7
:101D70009093800080937F0012E10DC0833051F476
:101D8000911108C082E498E19093800080937F00D5
:101D900014E001C010E080E480936F001DC0883023
:101DA00059F0893019F49093840002C08A3039F0D8
:101DB0008AE790E010E006C084E890E002C08AE77D
:101DC00090E011E09093800080937F0005C01E8119
:101DD00080E880936F0007C08F81811104C08E81DD
:101DE000811708F4182F1093610030C080916F00A4
:101DF00087FF2CC08091690090916A00009739F4A8
:101E00008881998190936C0080936B0012C084301C
:101E1000910539F48881998190936E0080936D00CB
:101E200008C08115984128F0809169008F7339F0BE
:101E30000DC089919991CEDE0250E1F6F5CF8091E7
:101E400068008260809368001092610010928100A7
:101E50008091600084FF43C0809161008F3F09F44E
:101E60003EC0082F893008F008E0801B8093610095
:101E70008091710098E8892780937100002319F1FF
:101E8000E0917F00F091800080916F0086FF0BC091
:101E9000A2E7B0E084918D93319682E790E0800FC5
:101EA0008A13F8CF0CC0CF01A2E7B0E0FC0121916A
:101EB000CF012D9322E730E0200F2A13F7CFF093C4
:101EC0008000E0937F00602F82E790E0F1DC0C5F00
:101ED0000C3019F08FEF809361000093600084E173
:101EE00096B3987131F48150D9F710928200109214
:101EF0007C0001E0811100E080917000801739F0D2
:101F0000011103C01092670035DE009370008CE968
:101F100091E00197F1F78091680080FF11C0F8947B
:101F2000E0E0F8E1E054F10983E080935700E895A0
:101F30003097C1F710926A00109269008ADE789497
:101F40000091680001FF0BC08AE390E20197F1F76E
:101F5000809169008F7311F07CDE01C02EDE02FFDC
:101F600013C0B99882E291EA0197F1F7F894BB9A0D
:101F70001BBE15BA10925F02EAEFF7E1E4918E2FD3
:101F800081508E3FC0F019C01092680080916700A8
:101F90008D7011F0B99801C0B99A80916600909146
:101FA00067000196909367008093660080369A4E92
:101FB00008F47ACED6CFE1BF000020CC0DCFF89444
:021FC000FFCF51
:061FC2005AFF17FA400867
:0400000300001800E1
:00000001FF
